S01900006F70656E626C745F73746D3332663035312E7372656303
S31508000000002000202D1800087D1800087D1800081B
S3150800001000000000000000000000000000000000D2
S315080000200000000000000000000000007D18000825
S3150800003000000000000000007D180008E90800081C
S315080000407D1800087D1800087D1800087D1800082E
S315080000507D1800087D1800087D1800087D1800081E
S315080000607D1800087D1800087D1800087D1800080E
S315080000707D1800087D1800087D1800087D180008FE
S315080000807D1800087D180008000000007D1800088B
S315080000907D1800087D1800087D1800087D180008DE
S315080000A07D1800087D1800087D1800087D180008CE
S311080000B07D180008000000007D180008FC
S315080000BC10B5064C2378002B07D1054B002B02D024
S315080000CC044800E000BF0123237010BDC8000020BF
S315080000DC00000000C8180008044B10B5002B03D00C
S315080000EC0349044800E000BF10BDC04600000000EC
S315080000FCCC000020C8180008002243088B4274D391
S3150800010C03098B425FD3030A8B4244D3030B8B42FE
S3150800011C28D3030C8B420DD3FF22090212BA030C07
S3150800012C8B4202D31212090265D0030B8B4219D3E8
S3150800013C00E0090AC30B8B4201D3CB03C01A524108
S3150800014C830B8B4201D38B03C01A5241430B8B4250
S3150800015C01D34B03C01A5241030B8B4201D30B0339
S3150800016CC01A5241C30A8B4201D3CB02C01A524160
S3150800017C830A8B4201D38B02C01A5241430A8B4223
S3150800018C01D34B02C01A5241030A8B4201D30B020C
S3150800019CC01A5241CDD2C3098B4201D3CB01C01A26
S315080001AC524183098B4201D38B01C01A5241430930
S315080001BC8B4201D34B01C01A524103098B4201D31E
S315080001CC0B01C01A5241C3088B4201D3CB00C01A8B
S315080001DC524183088B4201D38B00C01A5241430803
S315080001EC8B4201D34B00C01A5241411A00D2014628
S315080001FC524110467047FFE701B5002000F006F89B
S3150800020C02BDC0460029F7D076E770477047C0464E
S3150800021C72B6704762B6704710B5FFF7F9FF10BD96
S3150800022C70B508E0461C4D1C0B78037000F009FCF1
S3150800023C300029002200541EA4B2002AF2D170BD47
S3150800024C10B582B000F052FA002801D102B010BDE8
S3150800025C00F0EEFD0028F9D000F0C0FB00F00AFB18
S3150800026C00F034FE0E4A9169012319439161926993
S3150800027C13400193019B00F03DFA0100C022802037
S3150800028C8005FFF7CDFF074A136803218B430B4301
S3150800029C136000F02FFA4468FFF7BCFFA047D5E7B8
S315080002AC001002400000014070B50500002401E072
S315080002BC0134E4B20C2C15D800F0C3FB63001B19EF
S315080002CC9A00094BD358AB42F2D862001219900027
S315080002DC054A121852689B189D42E9D2024B1B1804
S315080002EC187A00E0FF2070BDE018000870B505000C
S315080002FC00240C2C10D800F0A4FB63001B199A00E0
S3150800030C074B9B181B7AAB4202D00134E4B2F0E7D8
S3150800031C1300034A985801E00120404270BDC046BC
S3150800032CE018000870B5050000240C2C10D800F055
S3150800033C88FB63001B199A00064B9B181B7AAB4269
S3150800034C02D00134E4B2F0E7024B9B18586800E07F
S3150800035C002070BDE018000810B5CB0509D103685C
S3150800036C994208D002C080229200FFF759FF01205B
S3150800037C00E0002010BD0120FCE7F8B50700006876
S3150800038CFFF792FFFF2821D000F050FE00257F2DA5
S3150800039C13D8AB003A68D418FB185E6800F051FB0A
S315080003AC320000232100022000F090FE002806D11E
S315080003BC23689E4208D10135E9E7012400E00024B0
S315080003CC00F04CFE2000F8BD0024F9E70024F9E7FC
S315080003DC70B504000D000C4B984208D00B4B994293
S315080003EC07D0FFF7CAFF002804D1002408E0084C00
S315080003FC00E0054C29002000FFF7AEFF002801D0CD
S3150800040C200070BD0024FBE7E8020020002000084D
S3150800041CE4000020F0B5C64600B507000C00150030
S3150800042C1E004B0A5B029846036801330DD03B68E5
S3150800043C984505D041463800FFF7CAFF071E26D057
S3150800044C3B68E41A3C1904340CE04146FFF784FF78
S3150800045C0028ECD118E02B78237001340135013EC5
S3150800046C002E10D000F0EDFA3B1DE31A0A4A93420F
S3150800047CF1D98021890041443800FFF7A9FF071EEE
S3150800048C07D0041DE7E7012004BC9046F0BD002008
S3150800049CFAE70020F8E7C046FF010000F0B587B080
S315080004AC0C0000230593884206D80126032805D993
S315080004BC102C04D9002602E00026F7E70026012EA8
S315080004CC02D0300007B0F0BDFFF710FF0700200080
S315080004DCFFF70CFF05002000FFF724FF2D18013D40
S315080004ECED1B0135AD0AADB2002302930397013318
S315080004FC049300F09BFD0024AC4212D200F0A1FA42
S3150800050C05A902A800F054FE002809D1039B019303
S3150800051C8022D2009446634403930134A4B2EBE7D9
S3150800052C002600F09BFDCCE701235B42024A1360D0
S3150800053C024A13607047C046E4000020E802002017
S3150800054C70B504000E0015004A1E134B1B1A9A426E
S3150800055C01D9002070BDFFF7A7FEFF2818D0301967
S3150800056C0138FFF7A1FEFF2814D0630A5B020B4A79
S3150800057C934206D033002A0021000948FFF74AFFA8
S3150800058CE8E733002A0021000648FFF743FFE1E7B6
S3150800059C0020DFE70020DDE7FFFF00080020000849
S315080005ACE4000020E8020020F8B506000C004A1EFC
S315080005BC0C4B1B1A9A4201D90020F8BDFFF774FEA2
S315080005CC0500A0190138FFF76FFEFF2D06D0FF288E
S315080005DC06D001002800FFF761FFEEE70020ECE7E4
S315080005EC0020EAE7FFFF000800B583B0104B1B6834
S315080005FC01331BD00E4A536891688C466344D16804
S3150800060C8C46634411698C46634451698C46634431
S3150800061C91698C466344D2699B185B42019301AA83
S3150800062C04210448FFF78CFF03B000BD0120FBE74B
S3150800063CE8020020C02000080E4B1B680E4A126800
S3150800064C9B180E4A12689B180D4A12689B180D4A7D
S3150800065C12689B180C4A12689B180C4A12689B184D
S3150800066C0B4A12689B18002B01D0002070470120FA
S3150800067CFCE7C046002000080420000808200008F3
S3150800068C0C20000810200008142000081820000868
S3150800069CC020000810B50B4B1B68013304D0094861
S315080006ACFFF76BFE002809D0074B1B68013306D0F1
S315080006BC0548FFF762FE002800D0012010BD012076
S315080006CCFCE7C046E8020020E4000020004870471A
S315080006DC0020000810B5FFF727FF10BD10B5FFF76F
S315080006EC2FFF10BD10B5FFF75FFF10BD10B5FFF754
S315080006FCA3FF10BD10B5FFF7E9FF10BD10B5FFF746
S3150800070C73FF002800D110BDFFF7C4FFFBE70000FC
S3150800071C054BDB699B0604D5034B9B8C03700120A8
S3150800072C70470020FCE7C0460044004010B580B274
S3150800073C084B188500F0C6F80A300400054BDB692F
S3150800074C1B0605D400F07DF900F0BCF88442F5D2FE
S3150800075C10BDC0460044004010B588B0E1231B020A
S3150800076C019300230293039304930C220592069398
S3150800077C0793054C01A9200000F0DEFE2368012230
S3150800078C1343236008B010BD0044004070B5060042
S3150800079C0D00402904D82800FFF7C8FF00240BE0F9
S315080007AC8121074800F09BF8F5E700F04AF9305D1F
S315080007BCFFF7BCFF0134A4B2ABB29C42F5D370BDB3
S315080007CC7C19000870B506000D00264B1C78002C09
S315080007DC17D12548FFF79CFF012801D0200070BDD2
S315080007EC214B1B78013BDBB23F2BF7D800F06AF89C
S315080007FC1E4B186000221E4B1A700132194B1A70C8
S3150800080CECE71B4B1B7801331748C018FFF780FF22
S3150800081C040001280BD000F055F8144B1B68643300
S3150800082C98421CD900220F4B1A700024D6E7104B9D
S3150800083C1A780132D2B21A700B4B1B789A4201D035
S3150800084C0024CBE792B2084901313000FFF7E8FCE7
S3150800085C0022044B1A70064B1B782B70BEE700243B
S3150800086CBCE7C0462D050020EC040020300500200E
S3150800087C2E0500200022014B1A60704710E000E09C
S3150800088C10B5FFF7F7FF054B054A5A6000229A6028
S3150800089C05211960034B1A6010BDC04610E000E034
S315080008AC7FBB000034050020044B1B68DB0303D513
S315080008BC034A1368013313607047C04610E000E022
S315080008CC3405002010B5FFF7EFFF014B186810BD73
S315080008DC3405002010B5FFF7F5FF10BD704710B5AD
S315080008EC00F0AFF8FCE7000010B500F09FF80128FF
S315080008FC03D00B4B1B78012B00D010BDFFF7E2FF82
S3150800090C084B1B68084A12689B18F533FF33984244
S3150800091CF3D30022024B1A70FFF792FCEDE7C046A0
S3150800092C3C050020380500204005002010B5054B75
S3150800093C1B78012B00D010BDFFF7C4FF024B1860C3
S3150800094CF9E7C0463C0500204005002010B50122F9
S3150800095C034B1A70FFF7EAFFFFF7C6FF10BDC04638
S3150800096C3C05002010B5FFF757FC00F066F8FFF7BA
S3150800097C87FFFFF7AFFE00F00DF8FFF7E7FF10BD96
S3150800098C10B500F05EF8FFF78FFF00F00FF8FFF7D1
S3150800099CABFF10BD10B500F0CFF9FFF7DDFE002256
S315080009AC014B1A7010BDC046C000002000B583B0BC
S315080009BC6B46D91D0748FFF705FF012801D003B080
S315080009CC00BD0022044B1A706B46D979014800F019
S315080009DCD3F9F4E744050020C00000207047000056
S315080009EC10B5054B1B78002B02D000F0BDF910BDD5
S315080009FCC9B2FFF7CBFEF8E7C0000020044B1B7802
S31508000A0C013BDBB2022B01D9402000E000207047E5
S31508000A1CC0000020044B1B78013BDBB2022B01D92A
S31508000A2C402000E000207047C000002010B500F000
S31508000A3C91F9002800D0012010BD10B500F004FA79
S31508000A4C10BD10B500F005FA10BD00000022014BD0
S31508000A5C5A70704784050020034BFE22DA70187111
S31508000A6C0221BA3A995270478405002010B5054CF4
S31508000A7C00232370FFF7EAFFFF23E3700122BB3B39
S31508000A8CE25210BD84050020064BFF22DA700022C4
S31508000A9C1A71597859719A71DA711A720621443297
S31508000AAC995270478405002010B50020FFF7D4FF33
S31508000ABC10BD0000094BFF22DA70094A9A6400221D
S31508000ACC1A715A719A710721D971002119725972C2
S31508000ADC99720831442299527047C0468405002001
S31508000AEC801A0008044BFF22DA7042689A640121C6
S31508000AFC442299527047C0468405002010B531200F
S31508000B0CFFF7AAFF10BD000070B5084CFF23E37071
S31508000B1C002525716571FFF771FFA071E5712572C6
S31508000B2C657207224423E25270BDC0468405002034
S31508000B3C70B5FFF78BFF0D4C01252570FF23E3706D
S31508000B4CEF3B237100236371FFF758FFA071FFF782
S31508000B5C61FFE071FFF75EFF000A20726572A572ED
S31508000B6C08224423E252FFF7B5FD70BD8405002028
S31508000B7C70B505004478FFF741FF0138844211DC53
S31508000B8C6A780A4C201DA16CFFF74AFBFF23E37019
S31508000B9C6B78A26C94466344A3646B780133442245
S31508000BACA35270BD2220FFF757FFFAE784050020F1
S31508000BBC70B504004578FFF721FF0138854212DC31
S31508000BCC61680B4DA9646278281DFFF729FBFF2382
S31508000BDCEB706378AA6C94466344AB646378013310
S31508000BEC4422AB5270BD2220FFF736FFFAE7C04607
S31508000BFC84050020F8B505001700002406E02B78BC
S31508000C0CE418E4B20135FFF71CFF31004E1E00292B
S31508000C1CF5D13C600120F8BD10B5084CFF23E370F4
S31508000C2CE21D4168A06CFFF7E5FF20710023637194
S31508000C3CA37108224433E25210BDC0468405002035
S31508000C4C70B504000E4B9D6CFFF7D8FE411E621C56
S31508000C5C2800FFF743FD00280DD0094CFF23E3704D
S31508000C6CFFF7CCFE0138A36C9C466044A0640122B5
S31508000C7C4423E25270BD3130FFF7EEFEFAE7C04668
S31508000C8C8405002070B504004578FFF7B7FE0238D6
S31508000C9C854210DC134BFF22DA700121BB3A9952BC
S31508000CAC617800290BD1FFF729FD002814D13130C2
S31508000CBCFFF7D2FE10E02220FFF7CEFE0CE0094B20
S31508000CCC986CA21CFFF70AFD002806D06378054A23
S31508000CDC916C8C466344936470BD3130FFF7BCFE4F
S31508000CECFAE7C0468405002010B5094B9B6C416891
S31508000CFC1800FFF7F7FC002806D0054BFF22DA7020
S31508000D0C0121BB3A995210BD3130FFF7A5FEFAE71F
S31508000D1C8405002010B5FFF793FA034BFF22DA700F
S31508000D2C0121BB3A995210BD8405002010B589B231
S31508000D3CFFF756FE10BD0000054B00221A709A6488
S31508000D4C43215A5401315A529A705A707047C04608
S31508000D5C84050020034B1B78002B01D0012070471B
S31508000D6C0020FCE78405002000214323014AD154C6
S31508000D7C7047C0468405002010B50378FF2B04D0B5
S31508000D8C294A1278012A14D010BDFFF7D1FE432345
S31508000D9C254AD35C012B42D04423234AD15E002931
S31508000DACF2DD100001224323C2540330FFF7BEFFC5
S31508000DBCEAE73733DAB2352A2DD893001B4AD358CB
S31508000DCC9F46FFF7D5FEE2E7FFF7F2FEDFE7FFF7F0
S31508000DDC89FEDCE7FFF720FFD9E7FFF76BFED6E7BE
S31508000DECFFF762FED3E7FFF74FFED0E7FFF73EFEAD
S31508000DFCCDE7FFF725FFCAE7FFF744FFC7E7FFF77D
S31508000E0C83FEC4E7FFF770FFC1E7FFF783FFBEE772
S31508000E1CFFF774FEBBE72020FFF71EFEB7E710208E
S31508000E2CFFF71AFEB8E7C04684050020A819000883
S31508000E3C10B59023DB051B69DB0701D5002010BD17
S31508000E4C00F03CF80120FAE710B5642000F006F82B
S31508000E5C10BD10B500F008F810BD0000014B188045
S31508000E6C7047C046D005002010B5FFF72BFD0F4B79
S31508000E7C1B68984210D30E4B1B78002B0DD1012200
S31508000E8C0B4B1A70FF320B4B9A61FFF71BFD0A4B83
S31508000E9C1B881818054B186010BD0022044B1A70D5
S31508000EAC0132FF32034B9A62EFE7C046D4050020A5
S31508000EBCD205002000080048D005002080225200E8
S31508000ECC014B9A627047C0460008004810B5074B9C
S31508000EDC01214942196100221A61D960DA609962C6
S31508000EEC9A6200F077FC002010BDC0460010024044
S31508000EFC10B5040000F0AEF9FA218900FFF7FCF8EA
S31508000F0C00F04AF8002221000120404200F012F8B5
S31508000F1C002010BD10B5064A136810210B43136048
S31508000F2C0020FFF7E5FF00F007FC002010BDC046C7
S31508000F3C0020024070B5002811DB8308144DC0331D
S31508000F4C9B005C5903221040C000FC3216008640F8
S31508000F5CB44389010A40824022435A5170BDC0B23B
S31508000F6C0F230340083B9B0806339B00094A94460B
S31508000F7C63445D6803221040C000FF2422008240AF
S31508000F8C954389010C4084402C435C60E6E7C046D7
S31508000F9C00E100E000ED00E001380A4B98420FD85A
S31508000FAC094A50600948036A1B021B0AC021090634
S31508000FBC0B430362002393600733136000207047CA
S31508000FCC0120FCE7FFFFFF0010E000E000ED00E069
S31508000FDC10B50022044BDA61044A13690124234331
S31508000FEC1361018010BDC046D805002000200240C0
S31508000FFC0C4BDB68DB0613D50B4AD36902210B4372
S3150800100CD3611023074AD268520706D50649CA691E
S3150800101C01200243CA6104221343024AD360704773
S3150800102C0023EFE700200240D8050020084B1B6977
S3150800103C1B060BD5064B074A5A60074A5A601B69AA
S3150800104C1B0601D5012002E0002000E000207047B5
S3150800105C0020024023016745AB89EFCD034A13698B
S3150800106C80210B43136100207047C04600200240C4
S3150800107C70B50400FFF72EFC0500134BDB68DB0785
S3150800108C0AD5631CF9D0002C19D0FFF723FC401B9A
S3150800109C8442F2D2032011E00B4BDB689B0602D587
S315080010AC2022094BDA60084BDB68DB0603D4064BB7
S315080010BCDB685B0705D5FFF79BFF012070BD032096
S315080010CCFCE70020FAE7C04600200240F0B583B0E2
S315080010DC04000E0001921F00204B1B7E012B02D12F
S315080010EC022003B0F0BD01221C4B1A761C48FFF7F0
S315080010FCBFFF00282DD1012C06D0022C02D00425C6
S3150800110C00241BE00225FBE70125F9E72022D21A69
S3150800111C390091400A000199D940114389B28019C6
S3150800112CFFF756FF0E48FFF7A3FF0E4A1369012176
S3150800113C8B43136100280CD10134E4B2AC4208D2BB
S3150800114C60002301202252429A18DFD43900D1407C
S3150800115CE4E70022014B1A76C3E7C046D8050020FF
S3150800116C50C30000002002400022064BDA61064BF1
S3150800117C1A6904210A431A611A693C310A431A612D
S3150800118C7047C046D8050020002002400022064BB6
S3150800119CDA61064B1A6902210A431A6158611A69FF
S315080011AC3E310A431A617047D805002000200240D8
S315080011BC70B505000E00244B1B7E012B41D0012275
S315080011CC214B1A760368012B22D02048FFF750FFD3
S315080011DC002831D101235B4233606C680130AB685F
S315080011EC9B026A68944663449C4226D22000FFF709
S315080011FCCDFF1648FFF73CFF154A136902218B43AE
S3150800120C1361002816D18023DB009C466444E6E76C
S3150800121C0E48FFF72DFF002801D001200DE0FFF73F
S3150800122CA3FF0A48FFF724FF094A136904218B43D5
S3150800123C136102E0346000E001200022024B1A76AA
S3150800124C70BD0220FCE7C046D805002050C300003C
S3150800125C00200240014B18687047C046C4000020A5
S3150800126C9023DB0598420DD0244B984216D0244B7C
S3150800127C98421FD0234B984228D0234B984231D002
S3150800128C00207047214B996A802292020A439A627F
S3150800129C9A6A1F490A409A620120F2E71B4B996A1F
S315080012AC8022D2020A439A629A6A1A490A409A62B8
S315080012BC0120E6E7154B996A802212030A439A62C3
S315080012CC9A6A15490A409A620120DAE70F4B996A1D
S315080012DC802252030A439A629A6A10490A409A6211
S315080012EC0120CEE7094B996A8022D2030A439A62F7
S315080012FC9A6A0B490A409A620120C2E70004004820
S3150800130C00080048000C0048001400480010024071
S3150800131CFFFFFDFFFFFFFBFFFFFFF7FFFFFFEFFFE1
S3150800132CFFFFBFFFF0B5002214E0866826408F68E1
S3150800133C6F433E43866024E0456A1B0A1C005C43E7
S3150800134C5C4363431C01E41AA5434C6963432B4372
S3150800135C436201320B681C00D44028D00124944007
S3150800136C2340F6D006681D005D436C006419E443FF
S3150800137C26404F686F433E4306604E68013E012E79
S3150800138CD3D9C66834400E696E433443C4604C687E
S3150800139C022CDED1FF2BCFD8046A5D436B431D01AB
S315080013ACED1AAC434D696B4323430362D1E74A6894
S315080013BC013A012A01D90120F0BDC96842689A434D
S315080013CC4B4313434360F6E730B5154B1A680120B7
S315080013DC02431A601968F825A94380242143196029
S315080013EC104A5A60104A1A601968104A1140196056
S315080013FC002159605A6BAA4322435A635A6B82439B
S3150800140C5A635A6B033082435A63D96219639868D4
S3150800141CBF22120402439A609960012030BDC0466F
S3150800142C001002400CF8FFF0FFFFF6FEFFFFFBFF73
S3150800143C044B5A6812090F231340034AD35CD8404D
S3150800144C7047C04600100240881A0008044B5A68B8
S3150800145C120A07231340034AD35CD8407047C04688
S3150800146C00100240981A000870B50B4B5B68802276
S3150800147C52021340934201D0084800E00848064D32
S3150800148CE96A0F2421400131FEF736FE6B689B0C86
S3150800149C1C400234604370BD0010024000093D0038
S315080014AC00127A0010B5054B5A680C231340082B0A
S315080014BC02D1FFF7D9FF00E0014810BD0010024029
S315080014CC00127A0010B50400FFF7ECFF2060FFF756
S315080014DCAFFF6060FFF7BAFFA06010BD10B500281B
S315080014EC23D1134B1A6B0323834013400206134371
S315080014FC022B13D0032B0BD0012B06D0FFF7D2FFF0
S3150800150CFFF796FFFFF7A2FF10E0FFF7CBFF0DE002
S3150800151C074B1B689B0709D5064807E0044B1B6A53
S3150800152C9B0703D58020000200E0002010BDC046B2
S3150800153C0010024000127A0030B585B004000D0088
S3150800154C0368DB0748D40368274A1A404B68C968FE
S3150800155C0B4329690B43A9690B431343036043687F
S3150800156C224A1340AA68134343608368204A1340EF
S3150800157C6A69134383601F4B984216D01E4B9842D8
S3150800158C17D0002000282AD02968002929D0AA6952
S3150800159C80231B029A4211D04B08C018FEF7ACFDEB
S315080015AC0004000CE060012017E00020FFF796FF0E
S315080015BCE8E701A8FFF786FF0398E3E740004B0826
S315080015CCC018FEF799FD0D4B034040080722104042
S315080015DC1843E060012000E0002005B030BD002073
S315080015ECFBE70020F9E7C046F369FFFFFFCFFFFFD3
S315080015FCFFFCFFFF0038014000440040F0FF0000EC
S3150800160C014B18607047C046C4000020114B1A687D
S3150800161C01210A431A605A680F4802405A601A6830
S3150800162C0E4802401A601A680D4802401A605A6839
S3150800163C0C4802405A60DA6A0F208243DA621A6B47
S3150800164C094802401A635A6B8A435A6300229A6005
S3150800165C7047C046001002400CB8FFF8FFFFF6FEB4
S3150800166CFFFFFBFFFFFFC0FFACFEFFFF10B52549D0
S3150800167C0B680122934313430B600B681A423CD048
S3150800168C214B19688022D2020A431A6019688022F3
S3150800169C52020A431A601C4B1B689B03FBD51A4B58
S315080016AC5A681A491140882252030A435A60DA6A60
S315080016BC0F218A43DA621968802252040A431A6097
S315080016CC114B1B689B01FBD50F4B5A68F0218A43BB
S315080016DC5A605A680E490A405A605A6803218A4366
S315080016EC01390A435A60084B5A680C231340082BD5
S315080016FCF9D10848FFF784FF10BD6A210648FFF7A1
S3150800170CEEF8BDE70020024000100240FFFFC2FFC2
S3150800171CFFF8FFFF006CDC02A01A000810B5FFF7F3
S3150800172CF9FBFFF7A3FF10BD10B5FFF7F7FFFFF79F
S3150800173C19F9FFF725F9FCE7F0B58BB0234B9A6935
S3150800174C01252A439A619A692A400392039A596990
S3150800175C80229202114359615969114002910299EA
S3150800176C5869802424032043586159692140019102
S3150800177C0199D9691143D961DB691A400092009B1A
S3150800178C80277F00049705950024069407940894EF
S3150800179C0F4E04A93000FFF7C5FDB76204950594F2
S315080017AC08949026F60504A93000FFF7BBFD0C2318
S315080017BC04930A3B059301330693079408940995F9
S315080017CC04A93000FFF7AEFD0BB0F0BD00100240C7
S315080017DC0008004810B5FFF7F7FD0D4880235B009D
S315080017EC8362FFF73DFD9020C005FFF739FD094BD5
S315080017FCD96909480140D9615969084A11405961A2
S3150800180C5A6902405A619A6901218A439A6110BD44
S3150800181C0008004800100240FFFFFDFFFFFFF7FF1E
S3150800182C0D4885460D480E490E4A002302E0D45849
S3150800183CC4500433C4188C42F9D30B4A0B4C0023FE
S3150800184C01E013600432A242FBD3FFF7DFFE00F07F
S3150800185C11F8FFF769FFFEE700200020C000002002
S3150800186CC8000020B41A0008C8000020F80500209B
S3150800187CFEE7000070B500260C4D0D4C641BA41039
S3150800188CA64209D1002600F019F80A4D0A4C641B29
S3150800189CA410A64205D170BDB300EB589847013683
S315080018ACEEE7B300EB5898470136F2E7AC1A000896
S315080018BCAC1A0008AC1A0008B01A0008F8B5C046ED
S315080018CCF8BC08BC9E467047F8B5C046F8BC08BCC0
S309080018DC9E4670475F
S315080018E00020000800080000040000000028000886
S315080018F0000800000500000000300008000800008D
S315080019000600000000380008000800000700000074
S315080019100040000800080000080000000048000811
S315080019200008000009000000005000080008000038
S315080019300A00000000580008000800000B0000001C
S3150800194000600008000800000C000000006800089D
S31508001950000800000D0000000070000800080000E4
S315080019600E00000000780008000800000F000000C4
S315080019700080000800800000100000002E2E5C2E5B
S315080019802E5C2E2E5C2E2E5C536F757263655C4141
S31508001990524D434D305F53544D333246305C72736B
S315080019A03233322E63000000FE0D0008220E0008B6
S315080019B0220E00081C0E0008220E0008220E00083F
S315080019C0160E0008040E0008100E00080A0E00087D
S315080019D0220E0008220E0008220E0008220E000819
S315080019E0220E0008220E0008220E0008220E000809
S315080019F0220E0008220E0008220E0008220E0008F9
S31508001A00220E0008220E0008220E0008220E0008E8
S31508001A10220E0008220E0008220E0008220E0008D8
S31508001A20220E0008220E0008220E0008220E0008C8
S31508001A30220E0008220E0008220E0008220E0008B8
S31508001A40220E0008220E0008220E0008220E0008A8
S31508001A50E00D0008D40D0008CE0D0008DA0D0008C8
S31508001A60220E0008220E0008220E0008E60D0008C5
S31508001A70220E0008EC0D0008F20D0008F80D00080B
S31508001A804F70656E424C54000000000000000000D4
S31508001A900102030406070809000000000102030406
S31108001AA02E2E5C6D61696E2E630000003E
S30908001AACE50000083B
S30908001AB0BD0000085F
S30D08001AB40400000000127A008C
S7050800182DAD
